:10000000FE283B08A0003908A1000130A2006400CE
:100010002720031C1A28A20B0728FF30A007031C67
:10002000A107031CF9283230A2000728640027200A
:100030000318162858200830A30059202720A20CA6
:100040002128A30B1D2859200314220808003A0870
:100050008400380884178004841300053719380693
:10006000FF3E0800A6003A0884000930A7000310EC
:100070003E20A60CA70B382803143E288413B71D76
:100080004D2800083804371D380680008417000802
:100090003804031C38068000592800083804031C63
:1000A0003806371938068000841738098005592822
:1000B0003717370D0639A0006720A100A00A672076
:1000C000371FCB283713A0000230E220CB280030A6
:1000D0008A00200882070134753403341534003453
:1000E0003C340C34D934A3003A08840038099A20EF
:1000F0008413A3080319F928F030A50022088038DA
:10010000A400F030A5030319A5000319A3030319E4
:10011000F9288A289D20030120183808A21F3808D2
:10012000A20803190301A40F972880067E289828A7
:100130000000812884178005F9282108200403196C
:10014000A00A8030201AA1062019A106A018A10635
:10015000210DA00DA10DF92883169B001C141A086F
:10016000F92883169A001C1555309D00AA309D0071
:100170009C149C18B9281C11F928A301A200FF3077
:10018000A207031CA307031CF9280330A100DF30DA
:10019000CB20BF28A101E83EA000A109FC30031C30
:1001A000D428A0070318D128A0076400A10FD128E4
:1001B0002018DA28A01CDE280000DE280800031022
:1001C000A10CA00CFF3E0318DF282008F928A2008C
:1001D0000530A80023082102031DF0282208200270
:1001E000043003180130031902302805031DFF30C5
:1001F000F9288313031383126400080007309F005B
:1002000083161C308500860183123C30BC00BD0182
:100210000530C0000F30BF000330C600C301C70166
:100220006400851D1429012A0630BA000430B80084
:100230000630B7000D3032200A303220C5014508A3
:10024000AC20BE000630BA000430B8000630B7005B
:100250003E083220C50A640045087F3C031D312951
:10026000382964003E085A3C031D372938291F29C4
:100270000630BA000430B8000630B7000D30322026
:100280000A3032200630BA000430B8000630B70019
:100290000D3032200A303220433032206830322094
:1002A000613032206E3032206730322065303220AB
:1002B0002030322070303220723032206F303220C5
:1002C0006730322072303220613032206D3032207F
:1002D0003F30322020303220793032202F3032200F
:1002E0006E3032200D3032200A303220D524A7253E
:1002F0000530BA001030B8000630B7001030BB002F
:100300002730B9000120031C012AC80064004808F6
:10031000793C03198C29012A0630BA000430B80050
:100320000630B7000D3032200A30322045303220FE
:100330006E303220743032206530322072303220FC
:10034000203032206E30322065303220773032203B
:100350002030322070303220723032206F30322024
:100360006730322072303220613032206D303220DE
:1003700020303220663032206F3032206C30322014
:100380006C3032206F3032207730322065303220AE
:1003900064303220203032206230322079303220F6
:1003A000203032205A3032202E3032200D30322090
:1003B0000A3032205B242C24C5010530BA001030ED
:1003C000B8000630B7001620C200450883169B000F
:1003D00083124208B1200630BA000430B80006305B
:1003E000B70042083220640042085A3C031DF92934
:1003F000012AC50A640045087F3C031D002A012A22
:10040000DD29D126EE26C5014508AC20BE006400DA
:100410003E08613C031D0D2AB32364003E08623C84
:10042000031D132ABE2364003E08633C031D192AE2
:10043000CB2364003E08643C031D1F2AD8236400BC
:100440003E08653C031D252AE42364003E08663C03
:10045000031D2B2AEE2364003E08673C031D312A4E
:10046000FB2364003E08683C031D372A0724640010
:100470003E08693C031D3D2A142464003E086A3C82
:10048000031D432A1F2464003E086B3C031D492AB8
:100490002C2464003E086C3C031D4F2A3824640061
:1004A0003E086D3C031D552A452464003E086E3C01
:1004B000031D5B2A502464003E086F3C031D612A23
:1004C0005B2464003E08703C031D672A67246400B7
:1004D0003E08713C031D6D2A742464003E08723C82
:1004E000031D732A812464003E08733C031D792A8E
:1004F0008D2464003E08743C031D7F2A9924640007
:100500003E08753C031D852AA32464003E08763C02
:10051000031D8B2AAF2464003E08773C031D912AFB
:10052000BC2464003E08783C031D972AC82464005C
:100530003E08793C031D9D2AD52464003E087A3C80
:10054000031DA32AE22464003E08313C031DA92AAE
:10055000EF2464003E08323C031DAF2AFD246400F2
:100560003E08333C031DB52A0B2564003E08343C8D
:10057000031DBB2A192564003E08353C031DC12A12
:10058000272564003E08363C031DC72A3525640034
:100590003E08373C031DCD2A432564003E08383C05
:1005A000031DD32A512564003E08393C031DD92A76
:1005B0005F2564003E08303C031DDF2A6D25640082
:1005C0003E08203C031DE52A652664003E082F3CBA
:1005D000031DEB2A7B2564003E082E3C031DF12AF7
:1005E000892564003E082C3C031DF72A98256400E9
:1005F0003E083F3C031DFD2AA72564003E083D3C04
:10060000031D032BB62564003E082B3C031D092B5C
:10061000C42564003E08263C031D0F2BD225640030
:100620003E08283C031D152BE02564003E082A3CAB
:10063000031D1B2BEE2564003E08403C031D212BAF
:10064000FD2564003E08413C031D272B72266400F3
:100650003E08423C031D2D2B852664003E08433C8A
:10066000031D332B982664003E08443C031D392BA0
:10067000AB2664003E08453C031D3F2BBE266400AC
:100680003E08463C031D452B0F2764003E08483CAE
:10069000031D4B2BD12664003E08493C031D512B02
:1006A000962764003E084B3C031D572BEA26640046
:1006B0003E084C3C031D5D2BDB2664003E084D3C90
:1006C000031D632BD62664003E084E3C031D692B98
:1006D000012764003E084F3C031D6F2B0427640074
:1006E0003E08503C031D752B4E2764003E08513CCC
:1006F000031D7B2B502764003E08523C031D812BB9
:10070000522764003E08533C031D872B2A276400B0
:100710003E08543C031D8D2B3D2764003E08553C8C
:10072000031D932BEE2664003E08563C031D992BB7
:10073000F12664003E08573C031D9F2BE52664000C
:100740003E08583C031DA52BE02664003E085A3C99
:10075000031DAB2B012AC50A640045087F3C031D1D
:10076000B22B012A042A0B2638263D08A3003C0898
:10077000BE203D08A3003C08BE20080038260B26FA
:100780000B260B263D08A3003C08BE203D08A30015
:100790003C08BE20080038260B2638260B263D08CC
:1007A000A3003C08BE203D08A3003C08BE20080072
:1007B00038260B260B263D08A3003C08BE203D082A
:1007C000A3003C08BE2008000B263D08A3003C08FF
:1007D000BE203D08A3003C08BE2008000B260B26C7
:1007E00038260B263D08A3003C08BE203D08A30088
:1007F0003C08BE200800382638260B263D08A300FA
:100800003C08BE203D08A3003C08BE2008000B2683
:100810000B260B260B263D08A3003C08BE203D08F6
:10082000A3003C08BE2008000B260B263D08A300B1
:100830003C08BE203D08A3003C08BE2008000B2653
:100840003826382638263D08A3003C08BE203D083F
:10085000A3003C08BE20080038260B2638263D0899
:10086000A3003C08BE203D08A3003C08BE200800B1
:100870000B2638260B260B263D08A3003C08BE207D
:100880003D08A3003C08BE200800382638263D0855
:10089000A3003C08BE203D08A3003C08BE20080081
:1008A00038260B263D08A3003C08BE203D08A300C7
:1008B0003C08BE2008003826382638263D08A3000C
:1008C0003C08BE203D08A3003C08BE2008000B26C3
:1008D000382638260B263D08A3003C08BE203D08DC
:1008E000A3003C08BE200800382638260B263826F0
:1008F0003D08A3003C08BE203D08A3003C08BE20E4
:1009000008000B2638260B263D08A3003C08BE2015
:100910003D08A3003C08BE2008000B260B260B2632
:100920003D08A3003C08BE203D08A3003C08BE20B3
:10093000080038263D08A3003C08BE203D08A3005F
:100940003C08BE2008000B260B2638263D08A300D5
:100950003C08BE203D08A3003C08BE2008000B2632
:100960000B260B2638263D08A3003C08BE203D0878
:10097000A3003C08BE2008000B26382638263D0878
:10098000A3003C08BE203D08A3003C08BE20080090
:1009900038260B260B2638263D08A3003C08BE202F
:1009A0003D08A3003C08BE20080038260B26382648
:1009B00038263D08A3003C08BE203D08A3003C08A3
:1009C000BE200800382638260B260B263D08A3003B
:1009D0003C08BE203D08A3003C08BE2008000B26B2
:1009E00038263826382638263D08A3003C08BE2085
:1009F0003D08A3003C08BE2008000B260B26382625
:100A0000382638263D08A3003C08BE203D08A30038
:100A10003C08BE2008000B260B260B26382638265D
:100A20003D08A3003C08BE203D08A3003C08BE20B2
:100A300008000B260B260B260B2638263D08A300A4
:100A40003C08BE203D08A3003C08BE2008000B2641
:100A50000B260B260B260B263D08A3003C08BE20C8
:100A60003D08A3003C08BE20080038260B260B26B4
:100A70000B260B263D08A3003C08BE203D08A30022
:100A80003C08BE200800382638260B260B260B26ED
:100A90003D08A3003C08BE203D08A3003C08BE2042
:100AA00008003826382638260B260B263D08A300DA
:100AB0003C08BE203D08A3003C08BE2008003826A4
:100AC0003826382638260B263D08A3003C08BE20D1
:100AD0003D08A3003C08BE200800382638263826EA
:100AE000382638263D08A3003C08BE203D08A30058
:100AF0003C08BE20080038260B260B2638260B267D
:100B00003D08A3003C08BE203D08A3003C08BE20D1
:100B100008000B2638260B2638260B2638263D08DB
:100B2000A3003C08BE203D08A3003C08BE200800EE
:100B3000382638260B260B26382638263D08A300F3
:100B40003C08BE203D08A3003C08BE2008000B2640
:100B50000B26382638260B260B263D08A3003C081A
:100B6000BE203D08A3003C08BE20080038260B2606
:100B70000B260B2638263D08A3003C08BE203D0866
:100B8000A3003C08BE2008000B2638260B2638267A
:100B90000B263D08A3003C08BE203D08A3003C08EE
:100BA000BE2008000B2638260B260B260B263D08F8
:100BB000A3003C08BE203D08A3003C08BE2008005E
:100BC00038260B26382638260B263D08A3003C087D
:100BD000BE203D08A3003C08BE2008000B260B26C3
:100BE0000B2638260B2638263D08A3003C08BE20DD
:100BF0003D08A3003C08BE2008000B2638263826F6
:100C00000B2638263D08A3003C08BE203D08A30063
:100C10003C08BE20080064004708013C031D112E5B
:100C2000202E86140630BA000830B8006E30A200BC
:100C30004008732086103D08A3003C08BE20080031
:100C400086140130CA0064004A084602031C322E92
:100C50000630BA000830B8006E30A200533073205E
:100C6000CA0F232E86103D08A3003C08BE200800B2
:100C700064004708013C031D3E2E4D2E86140630AD
:100C8000BA000830B8006E30A2003F08732086100A
:100C90003D08A3003C08BE20080086140130CA00AD
:100CA00064004A084602031C5F2E0630BA00083072
:100CB000B8006E30A200FA307320CA0F502E861092
:100CC0003D08A3003C08BE2008003D08A3003C08E6
:100CD000BE203D08A3003C08BE203D08A3003C0800
:100CE000BE200800FA30BC00BD011530C0003F3006
:100CF000BF003C30C60064004708013C031D842E41
:100D00006030BC00EA30BD0008007830BC00BD0196
:100D10000A30C0001E30BF001E30C6006400470805
:100D2000013C031D972E3030BC007530BD0008001B
:100D30005430BC00BD010730C0001530BF000A3080
:100D4000C60064004708013C031DAA2E1030BC00F9
:100D50002730BD0008003C30BC00BD010530C0009C
:100D60000F30BF000330C60064004708013C031D7C
:100D7000BD2EB830BC000B30BD0008001830BC00E0
:100D8000BD010230C0000630BF000130C600640063
:100D90004708013C031DD02EE830BC000330BD00E5
:100DA0000800861706138612061208008613061717
:100DB000861206120800861306138616061208000D
:100DC000861306138612061608006400051DE92E18
:100DD000E52E080086140130C10008008610C1010C
:100DE000080064004308003C031D002F0130C900C7
:100DF00064000B3049020318002F0427C90FF82E96
:100E000008000130C30008000130C40064000D3048
:100E1000440203180E2F0F27C40F062F080064008A
:100E20004108013C031D252F0630BA000830B800E8
:100E30006E30A200D03073200630BA000830B800FF
:100E40006E30A200D1307320292F1330A3008830D8
:100E5000BE20080064004108013C031D382F063005
:100E6000BA000830B8006E30A200533073203C2F17
:100E70000330A300E830BE20080064004108013CB4
:100E8000031D4B2F0630BA000830B8006E30A200A8
:100E9000083073204D2F6430BD2008000614080070
:100EA000061008000130C7003C08A0003D08A10062
:100EB000A301FA30E720031D612F6030BC00EA3047
:100EC000BD003C08A0003D08A100A3017830E72048
:100ED000031D6E2F3030BC007530BD003C08A000F3
:100EE0003D08A100A3015430E720031D7B2F1030E3
:100EF000BC002730BD003C08A0003D08A100A301B4
:100F00003C30E720031D882FB830BC000B30BD00FB
:100F10003C08A0003D08A100A3011830E720031DF4
:100F2000952FE830BC000330BD000800C7013C0825
:100F3000A0003D08A100EA30A3006030E720031DB7
:100F4000A42FFA30BC00BD013C08A0003D08A10060
:100F50007530A3003030E720031DB12F7830BC007E
:100F6000BD013C08A0003D08A1002730A3001030BF
:100F7000E720031DBE2F5430BC00BD013C08A0007B
:100F80003D08A1000B30A300B830E720031DCB2F94
:100F90003C30BC00BD013C08A0003D08A10003306E
:100FA000A300E830E720031DD82F1830BC00BD0196
:060FB00008006300D92FC8
:02400E00543F1D
:1042000050005300440076007600760053005100C1
:0442100053005A00FD
:00000001FF
